:020000040000FA
:02000000B7291E
:020008003F2D8A
:10001000831203134208E1000130E2004308031990
:100020001528E20D6210FF3E0F286208E300E20986
:1000300080304207840062088005841362088005CE
:100040000800C920E830F4000330F500F601F7019C
:10005000D2204408F4004508F500F601F701FE201F
:10006000F30CF20CF10CF00CF313F30CF20CF10C9A
:10007000F00CF313F30CF20CF10CF00CF31370080A
:10008000E4007108E500C9204608F4004708F500BF
:10009000F601F701D2206408F4006508F500F601C6
:1000A000F7010330003E03195C28F40DF50DF60D41
:1000B000F70D7410FF3E5328FE207008E800710809
:1000C000E9007208EA007308EB000A30F40000301F
:1000D000F5006408F0006508F10087217008E4006D
:1000E0007108E50000307102031D782803307002AA
:1000F00003187B280800610884006B08003C031D7E
:100100008B286A08003C031D8B286908003C031DEE
:100110008B286808003C0318C6286308800465081B
:100120000319A228E601E70166086702031D9A2861
:10013000650866020318A228EC01A421E60A031947
:10014000E70A94286408EC00A42162088005650889
:100150000319BA28E601E70166086702031DB22801
:10016000650866020318BA28EC01A421E60A0319FF
:10017000E70AAC286408EC00A4210130E802031C63
:10018000E902031CEA02031CEB027D2862088005D9
:100190000800831203130030F0003230F100F20146
:1001A000F3010800831203132230FC00F801F90167
:1001B000FA01FB01FC030319EE280310FB0CFA0CF7
:1001C000F90CF80CF30CF20CF10CF00C031CDA280F
:1001D000FC030319ED28EF20DE28EF200800740847
:1001E000F80775080318750FF90776080318760FD6
:1001F000FA0777080318770FFB0708008312031329
:10020000FB01FA01F901F801E001730DF80D740822
:100210006321F30D0730FC00730D5D217408731C1E
:100220001329632114297521F30DFC0B0C29720D80
:100230005D217408731C1E2963211F297521F20D8D
:100240000730FC00720D5D217408721C292963219E
:100250002A297521F20DFC0B2229710D5D217408EC
:10026000721C3429632135297521F10D0730FC00FA
:10027000710D5D217408711C3F296321402975218E
:10028000F10DFC0B3829700D5D217408711C4A2991
:1002900063214B297521F00D0730FC00700D5D21A5
:1002A0007408701C5529632156297521F00DFC0B2B
:1002B0004E2970185C29EF200800F80DF90DFA0D91
:1002C000FB0DE00D0800F8027508031C750FF9021C
:1002D0007608031C760FFA027708031C770FFB02DF
:1002E0000301031C0130E0020800F8077508031839
:1002F000750FF90776080318760FFA0777080318C1
:10030000770FFB07030103180130E0070800831291
:100310000313F801F9011030FC00710DF80DF90D0F
:100320007408F8027508031C750FF90203189F2959
:100330007408F80775080318750FF9070310F00D16
:10034000F10DFC0B8D29080083120313EC03EC0361
:100350006C08003C0318B129EC0300000000000009
:10036000A82900000000000000000000080083121F
:1003700085010230860087018316D13081001B3051
:100380008500003086000030870005309F00831212
:100390000230860020308B0080309F000530C20084
:1003A0000230C3000820C801203084000530C0009E
:1003B000031726308D00031783160C1483120C08C4
:1003C0008D0A03138000840AC00BDB29A501B60146
:1003D000B701B801A801A901AA01BB018B1724220A
:1003E00003302502031CF0299930B000B100B2009F
:1003F000FC30A70028103030BD00E8233008031976
:10040000062A1130B002B102B202FB29A501013067
:100410002502031C072A0230B0004030B1007130C1
:10042000A7002810A5013030BD00E82303302502C5
:10043000031C132AA50101302502031C1B2AA90154
:10044000AA01A501B601452A1030C4000330C50039
:100450006430C6000030C7008316051183122120C6
:100460008316051583121E302E251730C400043064
:10047000C5006430C6000030C70083160511831222
:1004800021208316051583120800A819EA220823E3
:10049000003036020319502A04303602031D5C2A4C
:1004A0003823FE30A700391C942A3D088400000838
:1004B000F0390319A713942A01303602031D652A67
:1004C0002030BD00FD30A700942A02303602031D03
:1004D000732A1E233030BD003930A700103031029E
:1004E000031CA712942AFB302507031C502AF63060
:1004F0002507031C602AE0302507031C502ADB3047
:100500002507031C692ACB302507031C502AC63057
:100510002507031C602AB0302507031C502AAB3086
:100520002507031C692A502AE823481CA72A703093
:10053000C4000330C5006430C6000030C700831615
:10054000051183122120831605158312B82AC81CB1
:10055000B82AE030C4000630C500E830C6000330D9
:10056000C7008316051183122120831605158312F7
:10057000C801BB1FC22AB60A053036020319B601EC
:10058000B717D92A3B1FC62A5E23D92A3B1ED92A70
:1005900006302402031CD32A55302402031CD92A16
:1005A0008B138225D42A8B13A401A501A901AA01CA
:1005B0008B17BB01A81C452A8824A810A815013058
:1005C0002202031D452ACA2401302102031D452AA7
:1005D000DC24452AA811203084000530C000031710
:1005E00026308D0003130008840A03178C0083163D
:1005F0008C130C1555308D00AA308D008C148C187E
:10060000FF2A0C1183128D0A0313C00BF32A080072
:1006100083169F13831281309F0025251F151F19F4
:100620000F2B76301E020318172B28151C2B8A302F
:100630001E02031C1C2B28111F10080083169F1775
:10064000831289309F0025251F151F19252B1E0891
:10065000AB0083161E088312AC001F10AC253208B5
:10066000B100B10E3308B1043408B200B20E080074
:10067000B9012330051A5C2B2308B0002408B1000F
:100680002508B20039143008031D492B1230B00080
:100690005B2B12303002031C5B2BB91403195B2B4C
:1006A000B0000E303002031C5B2B103030020318F8
:1006B0005B2B0630B0023030BD0008008B130530D4
:1006C000B600B7132008AD002108AE002208AF0025
:1006D0002030BD00C130A700E823BB1BB72B3B1B5C
:1006E000792BBB1E752BDC246A2B3B1E6A2B09253C
:1006F0006A2B3130A700E823BB1B6A2B3B1B8A2BDC
:10070000BB1E842BCA24792B3B1E792BFD24792B0D
:100710002030BD000D30A700E823BB1B792B3B1B0D
:10072000992BBB1E952B88248A2B3B1E8A2BED24EC
:100730008A2B3823C230A700E823BB1B882B3B1B26
:10074000B72BBB1EAB2B233084008C252430230217
:100750000318A301992B3B1E992B233084001A25E3
:10076000F9302302031D992B2330A300992B382342
:100770003230A700E823BB1B992B3B1BD52BBB1E9C
:10078000C92B243084008C25603024020318A40176
:10079000B72B3B1EB72B243084001A25F9302402D6
:1007A000031DB72B5930A400B72B20082D02031DC1
:1007B000E12B21082E02031DE12B22082F02031931
:1007C000E22BA815B601A901AA01A5018B17080003
:1007D00005303602031DED2BBB013D088400A71F29
:1007E000F62B000E8700823086007924271FFD2B10
:1007F00000088700423086007924840AA71E052C51
:10080000000E8700223086007924271E0C2C000859
:100810008700123086007924840AA71D142C000E4C
:1008200087000A3086007924271D1B2C00088700CA
:10083000063086007924B71F2E2C3608C000C00A67
:100840000430C100C0030319282C0310C10D222C51
:10085000FF3087004108033E86007924A71C432C03
:10086000F030391C512C05303602031D3C2CB030C1
:10087000B91C512C7030512C3A1C512C7030B91CC1
:10088000512CB030512C0030271C512C0530360231
:100890000319502C4030A71D512C1030271F512C0C
:1008A0005030FF3A8700003086002925023086004C
:1008B000FF308700BC0803195F2CBC03712C831622
:1008C000F030870083120708F039F03ABB00831636
:1008D0000030870083123B080319712C9630BC004E
:1008E0002814053036020319782C281CE82B281010
:1008F000080029252925281D7F2C0230860002307A
:10090000BE002E250230860029252925292508002C
:10091000A20A2208A6000F30A6050A302602031DEF
:10092000932C0630A2079D24A60022082602031C51
:100930009A2C08000130A200080002302102031D99
:10094000B62C200E0F39A6000310A60DA60DA60783
:10095000A60D20080F3926070339031DB22C2008E5
:10096000031DB42C2830C92C2930C92C0430210295
:100970000319C82C063021020319C82C09302102A2
:100980000319C82C113021020319C82C3130C92C8D
:1009900030300800A10A2108A6000F30A6050A3051
:1009A0002602031DD52C0630A10713302102031C9B
:1009B000DB2C0130A1000800A00A2008A6000F309F
:1009C000A6050A302602031DE72C0630A007A0303A
:1009D0002002031CEC2CA0010800A2030319FA2C2E
:1009E0002208A6000F30A6052602031D08000630C7
:1009F000A20208009D24A2000800A103031D022DED
:100A00001230072D0F302102031D08000930A1000C
:100A10000800A003FF302002031D102D6630182DA2
:100A20002008A6000F30A6052602031D0800063088
:100A3000A002080080030008B5000F30B50535029C
:100A4000031D080006308002080016302A2D3430BD
:100A50002A2D6930BE00BE0B2B2D0800BE000030D1
:100A6000BF000000000000000000000000000000C7
:100A700000000000BF0B312DBE0B2F2D0800FD0024
:100A8000030E8301FE000A08FF008A010408ED003E
:100A90000B194B2D692D0B11AA0F4F2DA90A3530BB
:100AA0002A02031D692D0C302902031C692D013017
:100AB000BA06A901AA017225281438080319642D61
:100AC000B80B682DB713682DB71F682D0230B8001A
:100AD00098256D0884007F088A007E0E8300FD0E35
:100AE0007D0E0900253084008C2560302502031C12
:100AF0000800A501243084008C2560302402031CEA
:100B00000800A401233084008C2524302302031C18
:100B10000800A814A3010800800A0008B5000F30DF
:100B2000B5050A303502031D0800063080070800AD
:100B300004303602031DAB2D59302402031DA62DAF
:100B400057302502031CA62D4814AB2D250824047C
:100B5000031DAB2DC81408002B0E0F39F03EB10059
:100B6000B107E23EB200323EB4002B080F39B207A3
:100B7000B207B407E93EB300B307B3072C0E0F3931
:100B8000B307B407B30DB40DB409B40D2C080F3975
:100B9000B407B10D0730B0000A30B407B303031C2B
:100BA000CD2DB307B203031CD12DB207B103031C33
:0C0BB000D52DB107B003031CD92D08009F
:02400E00723FFF
:1042000043006F0070007900720069006700680069
:1042100074002000280043002900200032003000F4
:10422000300037002D00320030003100390020000E
:104230006200790020004D002E00590061006D00E1
:1042400061006D006F0074006F00FF001400090032
:0642500001000000000067
:00000001FF
